:030000000219FDE5
:03000B000200A848
:03002B000201616E
:03005B000202ECB2
:030073000202D9AD
:1000800002030406080C10182030406080040608A3
:100090000C10182030406080A0C00003070F1F051F
:1000A000050D050305030302C2AFC0D0C0E0206206
:1000B00014E5256009E473E525F4F58AD262D0E001
:1000C000D0D0D2AF3285268AC262E526F4603630BF
:1000D000682C20720DD0E0D0D0C282C286C287D2F6
:1000E000AF32C282C286C287206F13206510740AA5
:1000F000D5E0FDE57BB40104429001FE4280D0E0F2
:10010000D0D0D2AF32758A00C28DD26201FE01B763
:10011000306805206502D28201B73068052065028B
:10012000D28601B7306805206502D28701B7C28147
:1001300030680A2065077406D5E0FDD28201B7C297
:100140008330680A2065077406D5E0FDD28601B7C2
:10015000C29030680A2065077406D5E0FDD2870199
:10016000B7C2AFC2AD53E6EFC0D0C0E0D2D3D2AF7A
:10017000C2CEE52A6007207449152A21C278007989
:100180000020742EE580307E01F430E50278FF53C4
:10019000DACF207E0343DA20307E0343DA10C2D860
:1001A000C271E580307E01F430E50279FFC3E89941
:1001B00070CB306103752A18207403752A18885C87
:1001C000D27020740DE52B6004152B21D243DA0187
:1001D000C2D82070024145A85C206102C270207420
:1001E00031C3E894F0400374F0F8E8C4540F28F8E1
:1001F0007984B703024112C313C313872120080275
:10020000C313200A06C3C898F8411228F850037493
:10021000FFF8C3E895655003E565F88822E52D549D
:10022000066022206B1FE536C333C333F8E564C391
:1002300013C313F9C3952240028922E82522F5222F
:1002400050037522FF852224A824C3E5249561402C
:1002500002A8618825E56670024189C3E8AA669A0A
:100260005003E8FAE4F9EAC333FBE568F45B29409C
:100270000D2567F8E56760021567400B41890AC3E1
:10028000E5679A5002056778FF8826C26FC3E526A6
:1002900094F84002D26F20CF0AD0E0D0D043E610CD
:1002A000D2AD32C2CF053A7801E52A60053074023A
:1002B000152AC3E55C94014005755F0041CF756068
:1002C00000756900E55F2401F55F5003755FFFD09D
:1002D000E0D0D043E610D2AD32C2AF53E67F759284
:1002E000FA7593FFC260759104D2AF32C2AF53E684
:1002F000EFC2ADC0D0C0E0C0F0D2D3D2AFA8FBA94E
:10030000FCC2D8307102615353DACF207E0343DA46
:1003100010307E0343DA20D271E580307E01F42074
:10032000E502612A88278928A18053DACF207E033D
:1003300043DA20307E0343DA10C2D8C2713074022F
:10034000A16C7800E580307E01F430E502A16C8874
:100350005CA15453DACF207E0343DA20307E03437E
:10036000DA10C271206102812C53DACF207E034360
:10037000DA10307E0343DA20C2D8D2718857895808
:10038000C3E89555F8E99556F97B007E087A00C3D5
:10039000E8948CE994005005755B00811E882178F3
:1003A000A2E6A8216055C3E894C8E994005008E487
:1003B000D2E4FB7A0A61F9C3E89468E99401500831
:1003C000E4D2E3FB7A0F61F9C3E894D0E9940250D8
:1003D00008E4D2E2FB7A1E61F9C3E894A0E994052F
:1003E0005008E4D2E1FB7A3C61F9C3E89498E994BF
:1003F000085008E4D2E0FB7A787E00C3E89559FC07
:10040000E9955AFD30E70AECF42401FCEDF43400E0
:10041000FD755B00C3EC9AED9E5003755B01885936
:10042000895A8557558558567802A154C3E89527AF
:10043000F8E99528F9307C02A138307B02A13830E8
:100440007A02A131207502814FE9FDE8FC816EE955
:10045000C313F9E813F8307902A131E9C313F9E8BD
:1004600013F8307802A131E9C313FDE813FC2061D1
:0F0470002CC3EC941CED940240028185ED701EAC
:10047F00C3EC94C850180529E52970021529C3E566
:10048F0029940A5002A16C755C00D270A16CE52909
:10049F00600215297888E6F97400207F087896B9EC
:1004AF000302789EE624FAFEE43400FFC3EC9EFCC0
:1004BF00ED9FFD9208B90310A2085007207609D2CC
:1004CF007681D7307602C276A2085016B9030DECAA
:1004DF00F42401FCEDF43400FD0204F178007900FE
:1004EF00A138B90315EC33FCED33FDC3EC940AFCD2
:1004FF00ED9400FD50047C007D00C3EC94FFED945F
:10050F0000400678FF7900A138EC8572F0A4C5F0A1
:10051F00A2F733F87900400302055478FF790002FF
:10052F000554E9C313F9E813F8307C0EE96002783B
:10053F00FFC3E81338F8E43400F9C3E894FFE994F3
:10054F0000400278FF885CD270206102A16C741F9A
:10055F00F4552F4BF52FC274EB7002D274752A1815
:10056F00307403752A0A306102A18020740353DAB4
:10057F00FE207403752B06D0F0D0E0D0D0D2AD435F
:10058F00E6103279010205B079030205B0790A024B
:10059F0005B0791E0205B079640205B079C802056D
:1005AF00B07817E4D5E0FDD8FAD9F6227A147B7823
:1005BF000205D77A107B8C0205D77A0D7BB4020522
:1005CF00D77A0B7BC80205D7E573D5E001227902F4
:1005DF00E4C283D5E0FDD286D5E0FDC286D5E0FD2D
:1005EF00D283D5E0FDE920E002D28230E002D2874B
:1005FF00E573D5E0FDE920E002C28230E002C28758
:10060F007496D5E0FDD9C9EAF8D5E0FDD8FBDBB883
:10061F00C28322C37C007D0075F00005F0EA33FA37
:10062F00EB33FB50F6EB13FBEA13FAC3E9FFE8FEDB
:10063F00E89AF8E99BF95004EFF9EEF8B3EC33FCC4
:10064F00ED33FDD5F0DFEDF9ECF822E889F08A20E3
:10065F00D2D4F8A9F07B0030F70B7BFFF42401F81C
:10066F00E9F43400F9E88520F0A4ADF0F8E985202D
:10067F00F0A4AFF0FEED2EF974003FFA7C04C3EA4C
:10068F0013FAE913F9E813F8DCF48BF030F70AE802
:10069F00F42401F8E9F43400F9E889F0C2D4F8A998
:1006AF00F02222C3E54113F9E54013F8C3E544985E
:1006BF00F8E54599F9500CC3E89480E994FF40168A
:1006CF000206E9C3E8947FE9940050030206E97833
:1006DF007F79000206E9788079FF8849894A22E507
:1006EF00492546F8E54A3547F9854A20E4300701A0
:1006FF00F43548FA30E709C3EA94F04015020727AA
:10070F00C3EA940F500302072778FF79FF7A0F028D
:10071F000727780079007AF0C3E5249561500AC362
:10072F0074019524500B020745E54A20E70E020796
:10073F0045E54A30E706884689478A482278A5E684
:10074F00FAC3E54933F8E54A33F9D15AE930E70BF3
:10075F00C3E89480E994FF4013E17FC3E8947FE9F5
:10076F0094005002E17F787F7900E17F788079FFF4
:10077F00E820E715C3E52398F84009C3E894014042
:10078F00030207A678010207A6E8F424012523F83F
:10079F0040030207A678FF884B2278A6E6FAA847FF
:1007AF00A948D15AE930E70CC3E89401E994FF4016
:1007BF00160207DAC3E894FFE9940050030207DA40
:1007CF0078FF79000207DA780179FFE920E715C38E
:1007DF00E54B98F84009C3E89401400302080178FB
:1007EF0001020801E8F42401254BF8400302080137
:1007FF0078FF88242278FF20692879A1E76023E514
:10080F0041601F74FF8541F0848539F0306A0375AC
:10081F00F005A4F8C5F0600278FFC3E895645002B4
:10082F00A864886322C3E5409440E5419401E563E1
:10083F005003140145046002F5632202084D22752E
:10084F00E890227883E6FF30EDF9A8BDA9BE0570C8
:10085F00C3E57094084052757000E9FA79A0E7601B
:0F086F0044EA7007E571601B020886C3E89571C3
:10087E006010E5715006600C140208920460F902D3
:10088E000892E571F571C39467401B7561C0C394FE
:10089E00044013756180C39404400B756140C3948A
:1008AE0004400375610075BB0B22E561F46002051F
:1008BE0061E570B4070375BB1022743279A787F017
:1008CE00A4C5F0A2F733F8C3E895614002A8618889
:1008DE00228824882588268864227540007541F078
:1008EE0022C2AF75C820A8CCA9CDAA3A30CF010A32
:1008FE0075C824D2AFAB3BAC3C883B893CC3E89B6C
:10090E00F8E99C206908F930660221FE2158AD3DB8
:10091E008A3DF9EA9DFA600478FF79FFAE3EAF3F5B
:10092E008B3E8C3FA83BA93CC3E89EF8E99FF9C3D8
:10093E00E54113FBE54013FAE82AF540E93BF541A2
:10094E0050067540FF7541FF21A5AA40AB41AC4052
:10095E00AD417E047F02C3EB9404400D1E1FC3EB1A
:10096E0094084005206A021E1FC3ED13FDEC13FC14
:10097E00DEF7C3EA9CFAEB9DFBEF6009C3E913F9BE
:10098E00E813F8DFF7EA28FAEB39FB8A408B41507F
:10099E00067BFF8B408B41C3EB94025002D2663034
:1009AE0069047F0321D07892E6FFC3E53794824035
:1009BE00110FC3E53794A040010FC3EF9406400218
:1009CE007F057E02E541C4540FF9E541C454F0F8A9
:1009DE00E540C4540F28F8C3E89EFAE99400FB40A2
:1009EE0009C3EA9402EB940050047A02E4FB414AF4
:1009FE00AA40AB41EBC4FEEAC4540F4EFCC3EA9CC2
:100A0E00FAEB9400FBC3E813C313F8EA28FAEB34AD
:100A1E0000FB8A408B41C3EB94024002C26678020F
:100A2E00EBC4FE7B00EAC4540F4EFAC3EA98FA40B8
:100A3E0005C3940250027A027892E6FF30600241BA
:100A4E004A855192855293D26043E680C3E49AF868
:100A5E00E49BF930660241D6E8FAE9FBD3E913FDCF
:100A6E00E813FC88518952C3EF94036038EF20E0FD
:100A7E000DE82CF8E93DF9ECFAEDFB020A9FE828A7
:100A8E00F8E939F9C3E82402F8E93400F97AFE7B73
:100A9E00FFC3EF9403400E8A538B54884D894E8CBE
:100AAE004F8D50610A885389548A4D8B4E8C4F8DD1
:100ABE00503069127553F07554FF754FF07550FF35
:100ACE007551F07552FF610AE8FAD3E813FC8851AC
:100ADE00C3EF94036020EF20E007E82CF8ECFA4116
:100AEE00F6E8282402F87AFEC3EF940340088A53EE
:100AFE00884D8C4F610A88538A4D8C4FE568C333FD
:100B0E005002646BF5683060026114753402D26075
:100B1E0043E680E52D54066034A840A941C3E9138D
:100B2E00F9E813F8C3E913F9E813F8306904E92476
:100B3E0040F9C2AF53E67F759100C3E498F594E493
:100B4E0099F595759104D26043E680D2AF22D264B6
:100B5E00754300752000306C03752040020B7BD26C
:100B6E0064754300752040306C0375200078017960
:100B7E0001206620E52D54066002C2647914E54119
:100B8E00C313700104F8C39414400278143069043E
:100B9E00781B791B206010E543600C306903D53457
:100BAE0004D26D8125711C0543E5BF5440B520026A
:100BBE00810F30690908C3E89940011861A22064C9
:100BCE000A08C3E8994002617B61A2C264C2AF53B6
:100BDE00E67F7591003066127594007595F87591E3
:100BEE0004D26043E680D2AF617BE5417EFFC33322
:100BFE004005C3334001FEC3E49E759400F5956134
:100C0E00ECC3E53394015002617B306402617BD802
:100C1E0002812361A2C26DC2AF53E67F759100853A
:100C2E005394855495759104854D92854E93D2605B
:100C3E0043E680D2AFE52D54066008206A020533E4
:100C4E00020C61306D0D206C0A2064071581158130
:100C5E000215302278003064027801E53775F0070E
:0E0C6E00A4F9E5F028F5F0E9A2F013A2F113C5
:100C7C00A2F213F537C394785003753778C3E53770
:100C8C0095384008D265C282C286C2873060028124
:100C9C0098854F92855093D26043E68022207D1632
:100CAC00C2AF754202C283D281306202D287D2AF08
:100CBC0075AA23020E98C2AF754202C283D290303D
:100CCC006202D282D2AF75AA23020E9830724320F0
:100CDC007D20C2AF75420390013F757B08C287C26D
:100CEC0090306204D28681F6D283D2AF75AA2402E8
:100CFC000E98C2AF75420390013F757B08C282C249
:100D0C0081306204D286A116D283D2AF75AA210299
:100D1C000E98207D17C2AF75420390011AC287301E
:100D2C006202D286D2AF75AA24020E98C2AF754267
:100D3C000390011AC282306202D286D2AF75AA2108
:100D4C00020E98207D16C2AF754204C281D290303B
:100D5C006202D286D2AF75AA21020E98C2AF75423A
:100D6C0004C290D281306202D286D2AF75AA24021C
:100D7C000E98307243207D20C2AF75420590012E33
:100D8C00757B02C286C283306204D282A19CD2815E
:100D9C00D2AF75AA23020E98C2AF754205900150CE
:100DAC00757B01C286C283306204D287A1BCD2900B
:100DBC00D2AF75AA23020E98207D17C2AF754205DB
:100DCC00900110C286306202D282D2AF75AA230281
:100DDC000E98C2AF754205900124C2863062EBD2E8
:100DEC0087D2AF75AA23020E98207D16C2AF75422A
:100DFC0006C290D283306202D282D2AF75AA24028C
:100E0C000E98C2AF754206C281D283306202D2877D
:100E1C00D2AF75AA21020E98307243207D20C2AF4A
:100E2C00754201900150757B01C282C2813062040F
:100E3C00D287C142D290D2AF75AA21020E98C2AF0E
:100E4C0075420190012E757B02C287C290306204FC
:100E5C00D282C162D281D2AF75AA24020E98207DB3
:100E6C0017C2AF754201900124C282306202D28750
:100E7C00D2AF75AA21020E98C2AF75420190011033
:100E8C00C287306202D282D2AF75AA24C265229088
:100E9C00010E757B00C282C286C287C281C283C228
:100EAC0090C26222788076FF0876FF0876FF08767B
:100EBC00FF08760308760408760A0876030876019C
:100ECC00087601788C76010876FF0876FF0876FFA5
:100EDC000876FF0876FF0876030876FF0876FF0889
:100EEC0076FF0876250876D00876FA0876FA087622
:100EFC00040876FF08760108760008767A0876FFF3
:100F0C000876010876010876000876030876002238
:100F1C007887E6FFC272BF0302D2727888E6C39468
:100F2C00036008C27DE630E102D27DC27E7889E69C
:100F3C0030E102D27EC3EF94026008758E01D27349
:100F4C00020F54758E00C273227880E614900080D4
:100F5C009378A5F67881E6149000809378A6F678BD
:100F6C0086E61490008D9378A7F67886E6F539C35B
:100F7C0094025003753902789CE67538FFB402036D
:100F8C007538A0B4030375388278A3E61490009AE0
:100F9C0093F566D19B22227896E6FA7897E6FB7851
:100FAC0088E6B40305C3EB940EFB307F047A007B18
:100FBC00FFC3EB9AFCC3948250027C8275720005CD
:100FCC0072EC8572F0A4C3E5F0947D40F222D27FDE
:100FDC00F1A31205A11205A17A007B007C10120569
:100FEC0097E55C2AFA74003BFBDCF37C04C3EB133F
:100FFC00FBEA13FADCF7FEC27F120FA322757C000A
:10100C00757D00E5EF20E6037520000520903FFF7D
:10101C00E520146006901FFF1460009304600375B4
:10102C00EF167597DE7597AD7581C043FF8012057D
:10103C009275EF0675A900E5C7240220E70DF5218E
:10104C00E5B120E0068521C743B101120E9B7580E6
:10105C003175A4CE75F1FF75D4DF7590FE75A501C1
:0F106C0075F2E175D50075A60175E34075E201D7
:10107B00120E9BE4F8F6D8FD756801120EB012152E
:10108B008178988673753001C2AF1205AB1205BB20
:10109B001205A11205C21205A11205C91205A11252
:1010AB00169E1205AB1205AB1205A6C2AF757C00DE
:1010BB00757D0078FA79FA308507D9FBD8F7021CD1
:1010CB0000120F1C120F55120FA2120FA378988645
:1010DB0073120E9B75881075890275C8247591045F
:1010EB0075D84075A82275B80275E690759B80750A
:1010FB009D0075BF8075AB0075D10C75BC5975BB68
:10110B000B75E88075B201120592D2AF12084A75C1
:10111B00360053DACF207E0343DA20307E0343DAE6
:10112B001043DA01C2D8C2711205ABD2617B037ACC
:10113B000CE55B70077A0CDB030210B61205A120DD
:10114B0070030210B6C270E55CC3940240E1E52F58
:10115B00541F855E5DF55EB55DD5DAD5C26153DA98
:10116B00CF207E0343DA20307E0343DA10C2D8C28D
:10117B007178A2E67008D274E52F54E0F52FC27592
:10118B007529001205A6307409C3E529940A40029B
:10119B00D27512059778023074027800C3E55C981B
:1011AB0040F0C2AF1205BB1205BB1205BBD2AF128A
:1011BB0005AB754C007888E6B4030241BC12059769
:1011CB00788CE6C3940150030212BCE530C3940142
:1011DB0050030212BC757CA5757DF1207435C3E5F7
:1011EB005C94FF50030212BCC2AF1205D0D2AF12F7
:1011FB0005A6C3E55C940150EFC2AF1205BB120507
:10120B009C1205BBD2AF1205A6C3E55C94FF40E967
:10121B000217237F05D27F120FA31205A6C2AFC2FE
:10122B007F120FA3AE5CC3E55C947FD2AF5002413B
:10123B00CC120592C2AF1205D0D2AFDFD8120FDAA3
:10124B00C3EE94057897F61205AB1216A67F0AD259
:10125B007F120FA31205A6C2AFC27F120FA3AE5C03
:10126B00C3E55C947FD2AF50E4120592C2AF120576
:10127B00BB12059C1205BBD2AFDFD4120FDAEE24E2
:10128B00037896F6F87997E7C39482400398500653
:10129B00E824827897F61205AB1215C31216D512F5
:1012AB0005A6120FA3C3E55C94FF500221E00217C1
:1012BB0023757C00757D00C3E55C954C4003855C14
:1012CB004C1205A678017988E7B403027805C3E5CB
:1012DB005C98400221C0C2AF1205D01205D0120596
:1012EB00D0D2AF1205AB753000E4F531F5320531D4
:1012FB00E531F4703F0532789AE67819146012786C
:10130B003214600D787D14600878FA14600375321E
:10131B0000C3E53298401D120E9B120592153275D3
:10132B00310078998673C2AF1205D0D2AF78988608
:10133B00731205A612059CE52A700530740201B6DE
:10134B0078012074027806C3E55C9840A17888E6A2
:10135B00C3940360031205A6E52A70030210B6C2FC
:10136B00AF120E9BE4F522F523F524F525F526F5B2
:10137B0067D2AF7885E6C333F565E4F544F545F5FB
:10138B0046F547F548F570F52CF52DF537757008D2
:10139B0075BB1012059212084E30EDFDA8BDA9BE0B
:1013AB00E97001F8887112085275700875BB10123C
:1013BB000F1CC2AF7561FF1208C8852261852262BE
:1013CB00852263D2AF75220175240175250175261F
:1013DB0001856069756A017888E6B40307C27D30C0
:1013EB007602D27DD268D269753300120DF5120EDA
:1013FB00241208E81208EF1208E81208EF1208E8A6
:10140B00120B6D1206B1120C62120CA91208EF121C
:10141B000B5C306E031206B22066031208043066B2
:10142B0003120834120C62120CD81208EF120B6D57
:10143B00306E031206EE120C62120D4F1208EF12F1
:10144B000B5C306E0312074C120C62120D7E1208ED
:10145B00EF120B6D306E031207A9120C62120DF511
:0F146B001208EF12084E120B5C120C62120E24C4
:10147A001208521208EF30692F856461856462850B
:10148A006069756A0179187A0CC3E53399400CC210
:10149A0069D26A8A357561FF0214B2C3E55C9401A8
:1014AA00400302140B021538306A1D206C1AE53508
:1014BA00147006C26AD26B810BF535C3E55C9401E0
:1014CA00400302140B021538753600788279A4E7B6
:1014DA0060027803C3E55F985054307404E52A60CB
:1014EA004D7888E6B40317207D05207607A10830D9
:1014FA007602A108206C07D26C856461814A78F073
:10150A00306C058564617820C3E541985002810BEF
:10151A00306C1BC26CC27D307602D27DD26A7535C0
:10152A0012856461810B0536E55C6002A13B753664
:10153A0000C2AF120E9B7887E6FE7602120F1C7865
:10154A0087EEF6E4F522F523F524F525F526F5656B
:10155A00752C00752D00D2AF1205A6120E9B78A429
:10156A00E66006D282D286D287307409C3E5369401
:10157A0004400201B641F4901A0D7820121605E5CE
:10158A0020B45A0CA3121605E520B4A5030215A32C
:10159A00120EB01215C30215C2901A0378807B0A84
:1015AA00121605A308DBF9901A0F788C7B1912160C
:1015BA0005A308DBF9901A2822C2AF1216481216A0
:1015CA0025901A00740E12160AA3740712160AA39B
:1015DA00741512160A901A0378807B0A121609A348
:1015EA0008DBF9901A0F788C7B19121609A308DB0D
:1015FA00F912165B121639901A2822E493F622E69B
:10160A00438F01538FFDFFC3E583941C400122EFF2
:10161A00857CB7857DB7F0538FFE22438F02438FB7
:10162A0001857CB7857DB7901A0DF0538FFC229007
:10163A001A0D745AD10A901A0E74A5D10A227A3058
:10164A0079D07820901A40D105E520F709A3DAF776
:10165A00227A3079D0901A40E7D10A09A3DAF9221E
:10166A00AB74A875BB01027984BB02027985BB03FE
:10167A00027986BB04027992BB05027987BB06020E
:10168A0079A3BB0702799CBB08027988BB09027956
:10169A0089E8F7227C051205ABDCFB22C2AF1205F2
:1016AA00BB1205C21205C91205D012059C1205BB50
:1016BA001205C21205C91205D012059C1205BB12E9
:1016CA0005C21205C91205D0D2AF22C2AF1205D087
:1016DA001205C91205C21205BB12059C1205D012C9
:1016EA0005C91205C21205BB12059C1205D01205C6
:1016FA00C91205C21205BBD2AF22AE74AF75C2AF12
:10170A001205BB1205BB1205BB12059CDEF21205BF
:10171A00D012059CDFF8D2AF22D1A6D19ED19E75F8
:10172A007401757501757600F1047C05AD5C1205CE
:10173A00ABC3ED955C70F5C3E55C9401400AC3E563
:10174A005C94FF403202175FD16AB1C3D1A6C2AF1F
:10175A0075EF16D19EDCD50576C3E5769403500263
:10176A0080C6D19E0575E5741490009F93F808C34E
:10177A00E57598500280AED19ED19E0574C3E5747A
:10178A00940A5002809C120EB0B1C3C2AF75EF1614
:02179A00D19EDE
:0319FD00021009CC
:101A00000E0715FFFFFFFF03040A0301015AA5019A
:101A1000FFFFFFFFFF03FFFFFF25D0FAFA04FF01DE
:091A2000007AFF0101000300FF40
:101A4000234D5232355F3135412320202020202084
:101A500023424C48454C492346383530232020202A
:101A60002020202020202020202020202020202076
:101C0000C2AFC2D37597DE7597AD7581C075A90057
:101C100043FF80752438752503B1DB7529A5752A26
:101C2000F175E34043F12053A4DF75D4FFD2857DE5
:101C3000FA780379E67C10752200752300901DE880
:101C40007B0675249875250130850281482085081A
:101C5000D8FBD9F9DCF781BA308508D8FBD9F9DC93
:101C6000F781BAB19BE493A3C39A6004DDC381BA40
:101C7000DBDBB18D600281317B08E493FAA3B16EA6
:101C8000DBF87A30B16E752200752300B18DEAFC65
:101C9000EBFDC3ED94FE400EB18D8A278B28ED300D
:101CA000E0048A828B83B18D7AC270D8C3ED94FE32
:101CB000601950CEBD0029EC600F7520007521FF22
:101CC000752900752A000200008100A827A92808AC
:101CD00009D804D90281DDB191EAF281D10D81A642
:101CE000C3ED94035051EDA2E092007AC5C3E582A2
:101CF0009400E583941C508C200010438F02438F86
:101D0000018529B7852AB7F0300027A827A9280818
:101D100009438F01538FFDD804D902A132C3E58353
:101D2000941C4003A3A117E28529B7852AB7F0A325
:101D3000A117538FFC81827AC1BD030CE493A3FAEF
:101D4000B152DCF8B14A81828184AA22AB23B16E00
:101D5000EBFAEA6222752608C3E52313F523E52290
:101D600013F52250066323A0632201D526EAB1DBD6
:101D7000B1DB75260AEAF4200102D285300102C2E5
:101D800085B1DBC3134002C201D526EB22B191EA33
:101D9000FB208502A191308502A196752608AE240C
:101DA000AF25C3EF13FFEE13FEB1DFB1DBC3EA13C0
:101DB0003085024480FA30E703632201C3E5231330
:101DC000F523E52213F52250066323A0632201D5F3
:101DD00026D9E52265236523F52222AE24AF250E00
:101DE0000FDEFEDFFCD20122424C48656C693437BD
:061DF0003163F85006010A
:00000001FF
